:1000000000800010CD000000150300001703000061
:10001000190300001B0300001D0300000000000086
:100020000000000000000000000000001F030000AE
:10003000210300000000000023030000C1010000B4
:100040002703000027030000270300002703000008
:1000500027030000270300002703000027030000F8
:1000600027030000270300002703000027030000E8
:1000700027030000270300002703000027030000D8
:1000800027030000270300002703000027030000C8
:1000900027030000270300002703000027030000B8
:1000A00027030000270300002703000027030000A8
:1000B0002703000027030000270300002703000098
:1000C00027030000270300002703000001488047A2
:1000D00001480047650E00002111000040F21003A6
:1000E000C1F200031A780AB901201870704700BFE6
:1000F00040F20000C1F2000008B503682BB140F2E5
:100100000003C0F2000303B1984708BD82B0034664
:1001100000918DF807309DF90730002B11DA4EF66B
:100120000053CEF200039DF8072002F00F02A2F167
:100130000401009AD2B24FEAC202D2B20B441A763C
:100140000DE04EF20013CEF200039DF90710009A65
:10015000D2B24FEAC202D2B20B4483F8002302B0FB
:10016000704700BF00B583B00190019A6FF07F43E4
:100170009A4202D94FF001031FE04EF21003CEF273
:100180000003019A22F07F4202F1FF325A604FF0E1
:10019000FF304FF01F01FFF7B9FF4EF21003CEF210
:1001A00000034FF000029A604EF21003CEF20003FB
:1001B0004FF007021A604FF00003184603B000BD6D
:1001C00040F21403C1F200031B6803F1010240F284
:1001D0001403C1F200031A60704700BF84B001909D
:1001E00040F21403C1F200031B68039340F21403AE
:1001F000C1F200031A68039BC3EB0202019B9A42FF
:10020000F4D304B0704700BF00B583B040F20803D8
:10021000C1F200031A6844F6D353C1F26203A3FB90
:1002200002134FEA931303F1FF331846FFF79AFFC7
:100230004FF0000301932BE0019A41F28013C0F2CA
:10024000000353F82230DAB2019941F28813C0F268
:10025000000353F82130104619464FF0010200F018
:1002600011F9019A41F28013C0F2000353F82230D1
:10027000DAB2019941F28813C0F2000353F8213039
:100280001046194600F03EF9019B03F1010301936A
:10029000019B012BD0D94FF0000301932DE0019A6F
:1002A00041F28013C0F2000353F82230DAB2019910
:1002B00041F28813C0F2000353F82130104619466A
:1002C00000F00AF94FF4FF70FFF788FF019A41F23E
:1002D0008013C0F2000353F82230DAB2019941F2E0
:1002E0008813C0F2000353F821301046194600F07D
:1002F00009F9019B03F101030193019B012BCED965
:10030000C9E700BF82B001900091FEE782B0019082
:100310000091FEE7FEE7FEE7FEE7FEE7FEE7FEE709
:10032000FEE7FEE7FEE7FEE784B003468DF8073000
:100330004FF0000303939DF80730042B29D801A246
:1003400052F823F059030000650300007103000018
:100350007D030000890300004CF20003C2F2090390
:10036000039316E04CF22003C2F20903039310E05A
:100370004CF24003C2F2090303930AE04CF260031B
:10038000C2F20903039304E04CF28003C2F20903B2
:100390000393039B184604B0704700BF84B0034624
:1003A0008DF807304FF0000303939DF80730042BBE
:1003B00029D801A252F823F0CD030000D903000090
:1003C000E5030000F1030000FD0300004CF2000310
:1003D000C2F20903039316E04CF22003C2F20903B0
:1003E000039310E04CF24003C2F2090303930AE0C6
:1003F0004CF26003C2F20903039304E04CF2800361
:10040000C2F209030393039B184604B0704700BF70
:1004100084B003468DF807304FF0000303939DF836
:100420000730042B29D801A252F823F04104000020
:100430004D04000059040000650400007104000030
:100440004CF20003C2F20903039316E04CF22003BE
:10045000C2F20903039310E04CF24003C2F2090315
:1004600003930AE04CF26003C2F20903039304E031
:100470004CF28003C2F209030393039B184604B0B5
:10048000704700BF00B587B00291134602468DF851
:100490000F208DF807309DF80F301846FFF744FF06
:1004A00003460593059B002B14D09DF80730002BC5
:1004B00007D0059B1A68029B42EA0302059B1A605B
:1004C00008E0059B1A68029B6FEA030302EA030235
:1004D000059B1A6007B000BD00B585B003460091CA
:1004E0008DF807309DF807301846FFF71DFF0346CB
:1004F0000393039B002B02D0039B009A9A6105B0E3
:1005000000BD00BF00B585B0034600918DF80730EF
:100510009DF807301846FFF707FF03460393039B38
:10052000002B02D0039B009ADA6105B000BD00BF2A
:1005300000B585B003468DF807309DF807301846A2
:10054000FFF7F2FE03460393039B002B02D0039BAD
:100550005B6901E04FF00003184605B000BD00BF25
:1005600084B00291134602468DF80F208DF80730B3
:100570009DF80F30002B0AD19DF80730002B06D1D3
:1005800048F28003C4F20203029A1A612EE09DF839
:100590000F30022B0AD19DF80730002B06D148F20C
:1005A0008003C4F20203029A1A631FE09DF80F3021
:1005B000002B0AD19DF80730012B06D148F28003A9
:1005C000C4F20203029A5A6110E09DF80F30022B28
:1005D0000BD19DF80730012B07D148F28003C4F2FC
:1005E0000203029A5A6300BF00E0FEE704B07047BE
:1005F00084B00291134602468DF80F208DF8073023
:100600009DF80F30002B0FD19DF80730002B0BD138
:1006100048F28003C4F202035A68029B22FA03F3F1
:10062000DBB203F001033CE09DF80F30022B0FD149
:100630009DF80730002B0BD148F28003C4F202036F
:100640005A6A029B22FA03F3DBB203F0010328E0AB
:100650009DF80F30002B0FD19DF80730012B0BD1E7
:1006600048F28003C4F202039A68029B22FA03F361
:10067000DBB203F0010314E09DF80F30022B0FD121
:100680009DF80730012B0BD148F28003C4F202031E
:100690009A6A029B22FA03F3DBB203F0010300E043
:1006A000FEE7184604B0704782B0034600918DF80B
:1006B00007309DF80730002B06D148F28003C4F2C2
:1006C0000203009ADA600BE09DF80730022B06D196
:1006D00048F28003C4F20203009ADA6200E0FEE707
:1006E00002B0704700B585B00291134602468DF8FE
:1006F0000F208DF807309DF80F209DF80730104629
:1007000002991A46FFF7BEFE05B000BD00B583B0E2
:10071000034600918DF807309DF807301846009980
:10072000FFF7DAFE03B000BD00B583B003460091C9
:100730008DF807309DF8073018460099FFF7E2FE64
:1007400003B000BD00B583B003468DF807309DF8B7
:1007500007301846FFF7ECFE0346184603B000BD0D
:1007600000B585B00291134602468DF80F208DF832
:1007700007309DF80F209DF80730104602991A4661
:10078000FFF7EEFE05B000BD00B585B0029113463F
:1007900002468DF80F208DF807309DF80F209DF848
:1007A0000730104602991A46FFF722FF0346184603
:1007B00005B000BD00B583B0034600918DF8073049
:1007C0009DF8073018460099FFF76EFF03B000BD93
:1007D00000B587B00291134602468DF80F208DF8C0
:1007E00007309DF80F301846FFF79EFD034605932E
:1007F000059B002B14D09DF80730002B07D0059BDC
:100800001A69029B42EA0302059B1A6108E0059BF4
:100810001A69029B6FEA030302EA0302059B1A614D
:1008200007B000BD00B585B08DF807008DF8061043
:10083000ADF804208DF803309DF807301846FFF717
:10084000ADFD03460393039B002B40D09DF803307E
:10085000002B19D09DF80630002B0AD0039B5B8833
:100860009AB2BDF8043042EA03039AB2039B5A805D
:100870002DE0039B1B889AB2BDF8043042EA0303C3
:100880009AB2039B1A8022E09DF80630002B0FD00D
:10089000039B5B889BB21A46BDF804306FEA0303E2
:1008A0009BB202EA03039BB29AB2039B5A800EE00A
:1008B000039B1B889BB21A46BDF804306FEA030302
:1008C0009BB202EA03039BB29AB2039B1A8005B063
:1008D00000BD00BF00B585B08DF807008DF806108B
:1008E000ADF804208DF803309DF807301846FFF767
:1008F00055FD03460393039B002B40D09DF8033026
:10090000002B19D09DF80630002B0AD0039B5B8A80
:100910009AB2BDF8043042EA03039AB2039B5A82AA
:100920002DE0039B1B8A9AB2BDF8043042EA030310
:100930009AB2039B1A8222E09DF80630002B0FD05A
:10094000039B5B8A9BB21A46BDF804306FEA03032F
:100950009BB202EA03039BB29AB2039B5A820EE057
:10096000039B1B8A9BB21A46BDF804306FEA03034F
:100970009BB202EA03039BB29AB2039B1A8205B0B0
:1009800000BD00BF00B585B0134602468DF80720B4
:100990000A468DF80620ADF804309DF80730184659
:1009A000FFF7FCFC03460393039B002B0CD09DF840
:1009B0000630002B04D0039BBDF804205A8303E0CB
:1009C000039BBDF804201A8305B000BD00B585B0B7
:1009D000134602468DF807200A468DF80620ADF82A
:1009E00004309DF807301846FFF7D8FC0346039300
:1009F000039B002B0CD09DF80630002B04D0039BEA
:100A0000BDF80420DA8303E0039BBDF804209A8339
:100A100005B000BD00B585B002460B468DF8072035
:100A20008DF806309DF807301846FFF7B7FC0346EF
:100A30000393039B002B0BD09DF80630002B03D0B3
:100A4000039BDB8A9BB205E0039B9B8A9BB201E080
:100A50004FF00003184605B000BD00BF00B585B0DB
:100A60008DF807008DF806108DF805208DF80430FC
:100A70009DF807301846FFF7CBFC03460393039B12
:100A8000002B2FD09DF80430002B12D09DF806309B
:100A9000032B26D89DF806309DF8062003998A5C22
:100AA000D1B29DF8052041EA0202D1B2039AD15495
:100AB00018E09DF80630032B14D89DF806309DF8F9
:100AC000062003998A5CD2B211469DF805206FEA90
:100AD0000202D2B201EA0202D2B2D1B2039AD154D6
:100AE00000E000BF05B000BD00B585B08DF807007F
:100AF0008DF806108DF805208DF804309DF807302C
:100B00001846FFF785FC03460393039B002B33D065
:100B10009DF80430002B14D09DF80630032B2AD802
:100B20009DF806109DF80620039B13441B7CDAB247
:100B30009DF8053042EA0303DAB2039B0B441A74B2
:100B40001AE09DF80630032B16D89DF806109DF884
:100B50000620039B13441B7CDBB21A469DF805302C
:100B60006FEA0303DBB202EA0303DBB2DAB2039BF0
:100B70000B441A7400E000BF05B000BD00B585B09D
:100B8000134602468DF807200A468DF806208DF898
:100B900005309DF807301846FFF73AFC03460393EB
:100BA000039B002B0AD09DF80630032B06D89DF836
:100BB0000620039B13449DF805201A7605B000BD5E
:100BC00000B585B0134602468DF807200A468DF819
:100BD00006208DF805309DF807301846FFF718FC01
:100BE00003460393039B002B0AD09DF80630032B8A
:100BF00006D89DF80620039B13449DF805201A771C
:100C000005B000BD00B585B002460B468DF8072043
:100C10008DF806309DF807301846FFF7F9FB0346BC
:100C20000393039B002B0AD09DF80630032B06D8B4
:100C30009DF80620039B13441B7DDBB201E04FF0BF
:100C40000003184605B000BD4CF20003C4F20F03C8
:100C5000D3F888304FEA136303F00303032B40F00B
:100C6000AA804CF20003C4F20F03D3F80C3103F056
:100C70000303032B00F2F48001A252F823F000BF1B
:100C8000910C0000F50C00005B0D0000910C0000C1
:100C90004CF20003C4F20F03D3F888304FEA434309
:100CA0004FEA534303F1010241F20023C0F27A03F9
:100CB00003FB02F24CF20003C4F20F03D3F88830B6
:100CC0004FEA134303F0FF0303F10103B2FBF3F216
:100CD0004CF20003C4F20F03D3F8043103F0FF0316
:100CE00003F10103B2FBF3F240F20803C1F2000387
:100CF0001A60B6E04CF20003C4F20F03D3F8883058
:100D00004FEA43434FEA534303F1010243F20063C6
:100D1000C0F26E1303FB02F24CF20003C4F20F03A5
:100D2000D3F888304FEA134303F0FF0303F10103C4
:100D3000B2FBF3F24CF20003C4F20F03D3F8043118
:100D400003F0FF0303F10103B2FBF3F240F20803E7
:100D5000C1F200031A6000BF83E04CF20003C4F24A
:100D60000F03D3F888304FEA43434FEA534303F16C
:100D700001034FEA03424CF20003C4F20F03D3F81D
:100D800088304FEA134303F0FF0303F10103B2FB82
:100D9000F3F24CF20003C4F20F03D3F8043103F072
:100DA000FF0303F10103B2FBF3F240F20803C1F2C7
:100DB00000031A6055E04CF20003C4F20F03D3F8AD
:100DC0000C3103F00303032B4BD801A252F823F09C
:100DD000E10D00000D0E0000390E0000E10D0000D5
:100DE0004CF20003C4F20F03D3F8043103F0FF0305
:100DF00003F1010240F60013C0F23D03B3FBF2F22F
:100E000040F20803C1F200031A602AE04CF200032A
:100E1000C4F20F03D3F8043103F0FF0303F101021E
:100E200041F60033C0F2B703B3FBF2F240F208031D
:100E3000C1F200031A6014E04CF20003C4F20F0385
:100E4000D3F8043103F0FF0303F101034FF4004230
:100E5000B2FBF3F240F20803C1F200031A6000E0B3
:100E600000BF70474CF20003C4F20F034FF02002A2
:100E7000C3F8A0214CF20003C4F20F03D3F8A03151
:100E800003F02003002B09D04CF20003C4F20F033F
:100E9000D3F8A03103F04003002BF5D04CF200034F
:100EA000C4F20F034FF00302C3F804214CF2000315
:100EB000C4F20F034FF00002C3F8A8214CF2000364
:100EC000C4F20F034FF00002C3F8AC214CF2000350
:100ED000C4F20F034FF00102C3F80C214CF20003DF
:100EE000C4F20F0340F26302C0F20502C3F884208B
:100EF0004CF20003C4F20F034FF0AA02C3F88C2097
:100F00004CF20003C4F20F034FF05502C3F88C20DB
:100F10004CF20003C4F20F034FF00102C3F880202B
:100F20004CF20003C4F20F034FF0AA02C3F88C2066
:100F30004CF20003C4F20F034FF05502C3F88C20AB
:100F40004CF20003C4F20F03D3F8883003F080633F
:100F5000002BF5D04CF20003C4F20F034FF0030254
:100F6000C3F880204CF20003C4F20F034FF0AA0232
:100F7000C3F88C204CF20003C4F20F034FF055026B
:100F8000C3F88C204CF20003C4F20F03D3F888306E
:100F900003F04073002BF5D04CF20003C4F20F03B2
:100FA0004FF02302C3F8A4204CF20003C4F20F0355
:100FB0004FF0AA02C3F8AC204CF20003C4F20F03B6
:100FC0004FF05502C3F8AC204CF20003C4F20F03FB
:100FD0004FF00102C3F8A0204CF20003C4F20F034B
:100FE0004FF0AA02C3F8AC204CF20003C4F20F0386
:100FF0004FF05502C3F8AC204CF20003C4F20F03CB
:10100000D3F8A83003F48063002BF5D04CF2000332
:10101000C4F20F034FF00302C3F8A0204CF2000308
:10102000C4F20F034FF0AA02C3F8AC204CF2000345
:10103000C4F20F034FF05502C3F8AC204CF200038A
:10104000C4F20F03D3F8A83003F44073002BF5D09B
:101050004CF20003C4F20F0348F2DE72C0F22842E1
:10106000C3F8C4204CF20003C4F20F034FF0000297
:10107000C3F8C8214CF20003C4F20F0343F23A0252
:101080001A604EF60053CEF200034FF000029A6051
:10109000704700BF08B500F04BF8074800B1006882
:1010A000064901B109680022FFF7AEF8044B0BB105
:1010B000AFF30080FEE700BF00000000000000006A
:1010C0000000000080B51448144B21E05C6899686A
:1010D000DD688C420CD0002205E0A6180832D6E963
:1010E000008941E902898C460831AA42F5D101E024
:1010F00004EB050C1C696146002204E0083200265E
:10110000002741E902670831A242F7D114330138C0
:101110000028DBD1FFF7BEFF01000000B011000086
:1011200001498D460149084700800010C5100000A4
:1011300070B541F29C1641F29C15C0F20006C0F257
:101140000005761BB61006D0002455F82430013473
:101150009847A642F9D841F29C1541F2A016C0F278
:101160000005C0F20006761B00F012F8B61006D09B
:10117000002455F8243001349847A642F9D870BDB0
:101180000100000003000000000004000000000453
:10119000F8B500BFF8BC08BC9E467047F1000000DF
:1011A000F8B500BFF8BC08BC9E467047DD000000E3
:1011B00000000000D011000000000010100000002E
:0411C0000800000023
:0811C40008EFFF7F01000000AD
:1011D000000000000000000000E1F5050000000034
:00000001FF
